:100000000C9460010C9498010C9498010C94980144
:100010000C9498010C9498010C9498010C949801FC
:100020000C9498010C9498010C9498010C94181F4E
:100030000C94C71F0C942A1A0C9498010C949801E4
:100040000C9498010C9498010C9498010C94B21A99
:100050000C9498010C9498010C9498010C949801BC
:100060000C9498010C9498010C9498010C949801AC
:100070000C9498015404540480048004E804060598
:100080001E061E061105AA05BB05BB0534205B2014
:1000900053215B205321A720CA2053212121302145
:1000A000290026022702540055002A423A003B004C
:1000B0005F00600061004C003C003D005C005D00A2
:1000C0005E0056003E003F0059005A005B0057009A
:1000D000E000E200115062006300580029001E0099
:1000E0001F002000210042422B0014001A000800CB
:1000F000150017002B0004001600070009000A0075
:10010000E1001D001B00060019000500E000E200F0
:10011000105013000B002C00C05CC15C01000100FA
:1001200001000100010001000100010001000100C7
:1001300001000100010001000100010001000100B7
:10014000010001000100A9000100010001000100FF
:10015000A800AA0010035000720069006D0065003D
:100160005F004D00000010035000720069006D0038
:1001700065004B00420000000403090409023B0033
:10018000020100A0FA090400000103010100092195
:100190001101000122400007058103080001090444
:1001A0000100010300000009211101000122B60035
:1001B000070582032000011201000200000008521E
:1001C000504D5001000102000105010902A1018505
:1001D000020901A100050919012908150025019549
:1001E00008750181020501093009311581257F95C6
:1001F000027508810609381581257F9501750881EA
:1002000006050C0A38021581257F950175088106BF
:10021000C0C005010980A101850319012AB7001595
:100220000126B700950175108100C0050C0901A1D8
:1002300001850419012AA002150126A00295017565
:10024000108100C005010906A1018506050719E016
:1002500029E7150025019508750181020507190098
:1002600029EF1500250195F0750181020508190196
:100270002905950575019102950175039101C00548
:10028000010906A101050719E029E71500250195D7
:10029000087501810295017508810105071900297A
:1002A000FF150026FF009506750881000508190155
:1002B0002905950575019102950175039101C0000D
:1002C00011241FBECFEFD4E0DEBFCDBF04B603FEC6
:1002D00018C080918F0290919002A0919102B091EC
:1002E00092028730904BA740B04B59F410928F0286
:1002F000109290021092910210929202E0E0F8E3C4
:10030000099511E0A0E0B1E0E6EBF4E402C005904D
:100310000D92A638B107D9F722E0A6E8B1E001C0F6
:100320001D92AF38B207E1F70E94F1110C945922E7
:100330000C94000081E0089581E008950C949C01E4
:1003400008950C94A0011F93CF93DF9300D000D0A9
:100350001F92CDB7DEB749835A836B8330918901F1
:1003600089819A81311114C0662359F0222349F002
:100370000E946408182F682F89819A810E940408BE
:1003800003C00E943508182F69817A81812F04C02B
:100390000E94640869817A810F900F900F900F90EE
:1003A0000F90DF91CF911F910C94810FFC01262FAC
:1003B000408151816281738184810C94A30181E029
:1003C0000895CF93DF93EC0160E00E94D601BE0157
:1003D000DF91CF910C94A1010C94B5100C94B11045
:1003E00008950E94AE060E94F0012FEF84E39CE086
:1003F000215080409040E1F700C000000C94D81AD2
:100400000F931F93CF93DF938C0161E00E94D6017D
:10041000EC01B8010E949E01882309F444C0B80190
:10042000CE010E948A158823F1F1B801CE010E9405
:1004300076188823C1F1B801CE010E948A1688235C
:1004400091F1B801CE010E94D217882361F1F80121
:100450008281882309F1CB358DE5D807C1F050F4AE
:10046000C115FCE5DF0781F0CF3DDC45A9F40E9412
:10047000910D19C0CC35EDE5DE0761F0CD35DD45D8
:1004800059F40E94DA0C08C00E94F1010CC00E94CD
:10049000E30C02C00E94E60CC801DF91CF911F91CE
:1004A0000F910C949A0180E0DF91CF911F910F91F1
:1004B00008950E940D1A80E00E94BF150C947702E7
:1004C0000E94AE140E947A020C94131A08950C94A0
:1004D000660281E008950C9469020895CF93C82FB5
:1004E0000E9467028C2F0E946B02CF91089580E0DA
:1004F0000C946E020E94D2180C946E020E94D218C4
:1005000090918801891721F0809388010C946E02E4
:100510000895CF93DF93CDB7DEB72B970FB6F8943E
:10052000DEBF0FBECDBF4F83588769877A878B8721
:1005300061110E94260C9E012F5F3F4F86E0F9015A
:1005400011928A95E9F785E0FE013796D90101906D
:100550000D928A95E1F789819A814C815D81452BC5
:1005600031F09F3F31F491E08F3F19F403C091E0E7
:1005700001C090E090FF09C049815A816B817C8164
:100580008D819E810E94420B05C0C9010E94DF013E
:100590008111F2CF2B960FB6F894DEBF0FBECDBF00
:1005A000DF91CF910895FC01808191810E94A6087E
:1005B0000895CF93882309F4A4C0C82F8238C1F4CA
:1005C0000E94D21881FD9DC069E380910201909143
:1005D00003010E94C8190E94480C2FEF81EE94E09D
:1005E000215080409040E1F700C0000069E319C04D
:1005F000833801F50E94D21880FD83C063E58091A5
:100600000201909103010E94C8190E94480C2FEF2B
:1006100081EE94E0215080409040E1F700C000005E
:1006200063E580910201909103010E94D319CF915B
:100630000C94480C8438C1F40E94D21882FD61C029
:1006400067E480910201909103010E94C8190E9401
:10065000480C2FEF81EE94E0215080409040E1F76C
:1006600000C0000067E4DDCF8CEF8C0F813AD0F43E
:100670006C2F80910201909103010E9448198823F8
:1006800049F06C2F80910201909103010E94D319CF
:100690000E94480C6C2F80910201909103010E94EE
:1006A000C819C5CF80E28C0F883048F4C77081E04C
:1006B00001C0880FCA95EAF70E94090CB8CFEBE594
:1006C000EC0FE33040F4F0E0E95BFE4F808190E016
:1006D000CF910C940619E8E5EC0FE73150F4F0E007
:1006E000EE0FFF1FE75EFE4F80819181CF910C944A
:1006F0001C19CD3E30F08C2F0E947E12CF910C94AD
:100700005013CF910895882309F464C0823879F496
:100710000E94D21881FF5EC069E38091020190912E
:1007200003010E94C8190E94480C69E310C0833875
:10073000B1F40E94D21880FF4DC063E580910201A0
:10074000909103010E94C8190E94480C63E58091B2
:100750000201909103010E94D3190C94480C843833
:1007600079F40E94D21882FF35C067E480910201BB
:10077000909103010E94C8190E94480C67E4E7CFDA
:100780009CEF980F913A10F4682FE1CF90E2980F08
:10079000983050F4877091E001C0990F8A95EAF77C
:1007A000892F0E940F0CD9CF9BE5980F933020F42E
:1007B00080E090E00C94061998E5980F973120F4AA
:1007C00080E090E00C941C198D3E20F00E94D9121C
:1007D0000C94501308951F93CF93DF93182FEB01C0
:1007E0000E94D902209741F08FE99FE00197F1F72D
:1007F00000C000002197F6CF812FDF91CF911F918C
:100800000C948303893319F060E070E002C060E566
:1008100070E00C94EB03882321F00E94090C0C94E7
:10082000480C0895882321F00E940F0C0C94480C6A
:100830000895CF92DF92EF92FF920F931F93CF9381
:10084000DF937C01D62FC72FFC0112810581029511
:100850000F700E94FF0B8823B9F01123A9F08C2F91
:10086000807F803421F080E28D0F883068F08091A5
:10087000720282FD09C082E00E94A80C0E94FF0B58
:1008800091E0D82ED92601C0D12CCC2EC2948FE075
:10089000C8228C2D90E08C30910508F0CFC1FC016E
:1008A000E65CFF4F0C9404228C2F807FCF7088234E
:1008B00011F0C295C07F112399F0CC2309F4AAC18D
:1008C00080E28D0F883010F0D11104C08C2F0E946F
:1008D000090C03C08C2F0E94190C0E94480C9AC16D
:1008E0008D2F0E948303CC2309F4A8C180E28D0FD1
:1008F000883038F1DD2329F18C2F0E941F0C24C091
:100900008C2F807FCF70803211F0C295C07FDD23A5
:1009100019F0D130A1F13DC08091720282FF17C061
:10092000112349F0CC2329F08C2F0E94090C0E943E
:10093000480C80E070C180E00E948303CC2309F45E
:100940007DC18C2F0E940F0C0E94480C77C111238F
:1009500071F0002341F0013031F40E94290C8C2BFE
:100960000E94310C6BC10E94290C8C2B1DC00023EE
:1009700019F0013009F462C10E943E0C25C0112318
:1009800021F0063008F05AC10EC0053008F056C1FB
:100990001BC0112361F0002331F0F701858180FF36
:1009A00039C18F7085838C2F0E940B0447C10023AF
:1009B00059F0D93309F03FC1FFEF07EE13E0F150D2
:1009C00000401040E1F735C18C2F0E94120436C15F
:1009D0008C2F86958695837019F0813061F02EC139
:1009E000112321F08D2F9C2F937002C080E090E0A6
:1009F0000E9406192BC1112321F08D2F9C2F93707B
:100A000002C080E090E00E941C1920C18D2F1123AC
:100A100019F00E947E1202C00E94D9120E94501347
:100A200015C18C2F837009F047C011110BC12D2FF8
:100A3000229526952770220F220F6D2F6F70862F1B
:100A400090E0A0E0B0E0022E04C0880F991FAA1F1A
:100A5000BB1F0A94D2F7D4FF10C04FE050E060E013
:100A600070E004C0440F551F661F771F2A95D2F708
:100A7000409550956095709503C040E050E0BA01F4
:100A8000C695C695C3708A019B01082B192B2A2B8A
:100A90003B2BC901B801C23049F058F4C13019F0FC
:100AA0000E941A07CFC00E940807CCC00E942C07E2
:100AB000C9C00E940607C6C0112319F08C2F81708F
:100AC00001C08695882309F4BDC02D2F2295269557
:100AD0002770220F220F6D2F6F70862F90E0A0E0FD
:100AE000B0E0022E04C0880F991FAA1FBB1F0A94F2
:100AF000D2F7D4FF10C04FE050E060E070E004C0D7
:100B0000440F551F661F771F2A95D2F740955095C1
:100B10006095709503C040E050E0BA01C695C69557
:100B2000C3708A019B01082B192B2A2B3B2BC9016F
:100B3000B801C23049F058F4C13019F00E94DF0703
:100B400081C00E94CD077EC00E94F1077BC00E9439
:100B5000400778C0CF70112339F08C2F0E946607B0
:100B60008D2F0E940B046EC08D2F0E9412048C2FBB
:100B70000E94870767C0D23F21F128F4D03F41F09F
:100B8000D13FC1F043C0D33F19F1D43F79F03EC00B
:100B9000112341F0053008F051C08C2F8F710E9455
:100BA000AC074CC0063008F049C0F7CF8091720204
:100BB00082FF18C0112339F08C2F8F710E946607B5
:100BC0003DC01123C9F38C2F8F710E94870736C057
:100BD000112329F08C2F8F710E9451072FC00E9482
:100BE0004C072CC0112349F0CF718C2F0E9466074F
:100BF00063E08C2F0E948D0C21C081E00E94A80C24
:100C00000230E0F082E00E94A80C18C0112331F0FD
:100C1000002391F28D2F0E94D90210C0002399F277
:100C2000D93349F41FEF27EE33E011502040304014
:100C3000E1F700C000008D2F0E94830388EF8C0D28
:100C4000843020F40E94D2180E946E02DD20C9F088
:100C50000E94FB0B80FD15C0F70112820E94F50B6C
:100C60000E946607C7010E9462060E94F50BDF9191
:100C7000CF911F910F91FF90EF90DF90CF900C9448
:100C80008707DF91CF911F910F91FF90EF90DF9039
:100C9000CF9008950F931F93CF93DF93EC0168815A
:100CA00079818A810E94B1088C010E9403080E9408
:100CB000F406B801CE010E941904DF91CF911F9173
:100CC0000F910895CF93DF93EC01988189812B8157
:100CD0003C81232B31F08F3F31F481E09F3F19F4A9
:100CE00003C081E001C080E080FD1DC0CE010E94F4
:100CF0000002811110C00E94FF0B8823A1F08A819D
:100D0000882389F08091720282FD0DC082E0DF911C
:100D1000CF910C94A80CCE010E944A06CE01DF911F
:100D2000CF910C94E101DF91CF91089580E090E0A4
:100D30000E94061980E090E00E941C190E94260C77
:100D40000E94480C0E948F140C9450138091020151
:100D5000909103010E94DE190C9496060E94160CD5
:100D60000C94A60692959F70963079F010F49250EC
:100D700001C09A50923068F4803F69F018F4883EC0
:100D800040F409C0843F29F406C0883E20F0813F2A
:100D900011F080E0089581E00895FC018081918147
:100DA0000E94A6080E94B2060895CF93DF9300D058
:100DB00000D01F92CDB7DEB70F900F900F900F901D
:100DC0000F90DF91CF910895CF93DF9300D000D0A3
:100DD00000D0CDB7DEB726960FB6F894DEBF0FBEB3
:100DE000CDBFDF91CF910895089508950C94F50635
:100DF0000C94F6060E94F8066093A2017093A3017A
:100E00008093A4019093A5010C9496060C94FA0685
:100E10000F931F930091A2011091A3012091A401AF
:100E20003091A501602B712B822B932B1F910F9179
:100E30000C94FA060F931F930091A2011091A30145
:100E40002091A4013091A501602371238223932373
:100E50001F910F910C94FA060F931F930091A2011A
:100E60001091A3012091A4013091A5016027712761
:100E7000822793271F910F910C94FA060C94F50684
:100E80000E943E0760939E0170939F018093A00192
:100E90009093A1010C94960660E070E0CB010C9455
:100EA00040070F931F9341E050E060E070E08A013B
:100EB0009B0104C0000F111F221F331F8A95D2F718
:100EC000C901B8011F910F910C9440070F931F9314
:100ED00041E050E060E070E004C0440F551F661F21
:100EE000771F8A95D2F780919E0190919F01A091E2
:100EF000A001B091A1018A019B01082B192B2A2B7B
:100F00003B2BC901B8011F910F910C9440070F931F
:100F10001F9341E050E060E070E004C0440F551FB3
:100F2000661F771F8A95D2F740955095609570950A
:100F300080919E0190919F01A091A001B091A1018B
:100F40008A019B01082319232A233B23C901B801E5
:100F50001F910F910C9440070F931F9341E050E0B5
:100F600060E070E004C0440F551F661F771F8A952C
:100F7000D2F780919E0190919F01A091A001B09124
:100F8000A1018A019B01082719272A273B27C901AC
:100F9000B8011F910F910C9440070F931F9300917C
:100FA0009E0110919F012091A0013091A101602B21
:100FB000712B822B932B1F910F910C9440070F9351
:100FC0001F9300919E0110919F012091A0013091EB
:100FD000A10160237123822393231F910F910C940D
:100FE00040070F931F9300919E0110919F01209144
:100FF000A0013091A10160277127822793271F91BB
:101000000F910C9440070895282F362F892F66E002
:101010000E948721820F982F9770A1E001C0AA0F2C
:101020009A95EAF786958695869590E065E070E05A
:101030000E949021FC01E657FE4F40E050E0632FF4
:1010400070E090819B01042E02C0369527950A948A
:10105000E2F72170219529272A23292721934F5F21
:101060005F4F4530510569F70895282F892F66E0B5
:101070000E948721820FA82FA77086958695869556
:1010800090E065E070E00E949021BC0140E050E0FB
:1010900080E0FB01E40FF51FE657FE4F208130E0B2
:1010A0000A2E02C0369527950A94E2F7217033275D
:1010B000042E01C0220F0A94EAF7822B4F5F5F4F84
:1010C0004530510531F70895BF92CF92DF92EF92EC
:1010D000FF920F931F93CF93DF938C01C0909E01DB
:1010E000D0909F01E090A001F090A1018091A20119
:1010F0009091A301A091A401B091A501C82AD92A79
:10110000EA2AFB2ACFE1D0E0D701C6010C2E04C0A9
:10111000B695A795979587950A94D2F780FD04C058
:10112000219790F7B12C07C0BC2EB8018C2F0E94DC
:101130009C0F0197A9F38B2DDF91CF911F910F91F8
:10114000FF90EF90DF90CF90BF900895CF93DF9303
:10115000EC010E946408BE010E949C0FDF91CF91B8
:1011600008951F93CF93DF93EB0190918901992309
:1011700021F0CB010E94A60813C0882349F0CB01BF
:101180000E946408182F682FCE010E94040804C032
:10119000CB010E943508182FBE01812F0E949C0FA1
:1011A000DF91CF911F910895CF93DF93C091A60156
:1011B0008091A701C817A1F0D0E0CE0166E070E0F1
:1011C0000E949021FC01E855FE4F408151816281CF
:1011D0007381848195810E94E4062196C770E8CFCF
:1011E000DF91CF9108954091D8015091D90160913C
:1011F000DA017091DB018091DC019091DD010C94AA
:10120000E406FF920F931F93CF93DF938091DD014C
:1012100082958F7009F062C08091DA01882309F409
:101220005DC02091A601F090A7011091D801009116
:10123000D901A091DB01B091DC0181E01F3F09F0F1
:1012400080E0C0910001D0910101482F2F1509F4D1
:1012500045C0109721F00F3F21F080E003C081E0EE
:1012600001C0842F30E080FD35C0C90166E070E028
:101270000E949021FC01E855FE4F818180132AC015
:101280008081811327C08281811124C08381948150
:101290008A1B9B0B8C179D07E8F48091DD018F70F2
:1012A00080618093DD01C90166E070E00E949021B9
:1012B000FC01E355FE4F90819F709061908388ED13
:1012C00091E00E946206DF91CF911F910F91FF90F4
:1012D0000C94D4082F5F3F4F2770B8CFDF91CF9188
:1012E0001F910F91FF9008959F92AF92BF92CF925E
:1012F000DF92EF92FF920F931F93CF93DF93CDB7BF
:10130000DEB761970FB6F894DEBF0FBECDBF8C017C
:1013100085E0F801DE011D9601900D928A95E1F7B6
:10132000F801E2809091D8013091D9016091DB0100
:101330007091DC016115710531F03F3F31F481E0BE
:101340009F3F19F403C081E001C080E0F82FF170E5
:101350009F2E80FD47C1F80140812181A380B48088
:1013600088EDC82E81E0D82EF090DA01F501E61B59
:10137000F70B6091000170910101FF2009F4DCC0BE
:101380008091DD01582F507FE617F70708F096C0CF
:10139000511155C0231313C0491311C0FE2CE11085
:1013A0000EC08F7080618093DD010E94F308C6013A
:1013B0000E9462068091DD01F801858350C1AB284F
:1013C00031F02F3F31F481E04F3F19F403C081E049
:1013D00001C080E080FD03C081E08E2502C080E076
:1013E00090E0F82FF170FF2E80FF1FC0E091A60162
:1013F0003091A701E31709F410C1F0E0CF0166E0D6
:1014000070E00E949021DC01A855BE4F11968C918E
:101410001197281307C08C91481304C012968C9121
:10142000E81203C03196E770E5CFFE2CEE2009F4F8
:1014300016C18091DD0181608093DD0154C02313CA
:1014400006C0491304C0E11002C0F80199C0C801E8
:101450000E94CD06882361F1EE2051F12091DD013B
:10146000822F82958F7090E0029774F08091D8015E
:101470009091D90198878F831986BB86AA862C877D
:10148000CE0107960E94620686E0F801A8EDB1E061
:1014900001900D928A95E1F70E9401090E94F308DC
:1014A0000AC0231711F1C8010E94CD0681112CC07A
:1014B000C8010E946206FF24F394D1C05111F1CFFC
:1014C0007A2DB98AA88A522F6E2D89890E94D50655
:1014D00088ED91E00E94620686E0F60111928A95FD
:1014E000E9F70E94F308F12CBAC04913DCCFE110F0
:1014F000DACFF8018583C8010E94620686E0F60112
:1015000011928A95E9F7ABC0EE2091F22091DD01AE
:10151000822F82958F7090E002970CF4B5CF809166
:10152000D8019091D9019A8389831B82BD82AC82B4
:101530002E83CE010196A6CFE617F70708F044C028
:10154000FE2CEE2009F4B4CF231330C049132EC073
:101550002091DD0120FD21C0822F82958F70482FC0
:1015600050E041155105C9F0F80125834F30510570
:1015700041F08F5F982F9295907F822F8F70892BEB
:101580008583C8010E94620686E0F801A8EDB1E0FB
:1015900001900D928A95E1F73DC086E0F801A8ED33
:1015A000B1E001900D928A95E1F759C0C8010E94FF
:1015B000CD06811169CF8091DD0181608093DD01CD
:1015C000C8010E9462064BC07A2DB98AA88A522FA0
:1015D0006E2D89890E94D50686E0F60111928A95C2
:1015E000E9F718C0EE2009F463CFC8010E94CD06C8
:1015F000F82E882309F45CCF86E0F801A8EDB1E06D
:1016000001900D928A95E1F788ED91E00E94D30256
:101610000E9401090E94F30822C04D872E878D8504
:101620009E850E94A608292F22952F70223028F42B
:101630009F7039F0811105C00BC0243028F49F70D1
:1016400049F4805E883020F0C8010E9462069F2C19
:10165000F92C05C0F8019581907F99F7F9CF8F2D6E
:1016600061960FB6F894DEBF0FBECDBFDF91CF916C
:101670001F910F91FF90EF90DF90CF90BF90AF90B0
:101680009F900895CF93DF93CDB7DEB72C970FB619
:10169000F894DEBF0FBECDBF4F83588769877A8726
:1016A0008B879C87CE0107960E9474098823D1F00E
:1016B0009F8188852A853B85232B31F08F3F31F42C
:1016C00081E09F3F19F403C081E001C080E080FD0C
:1016D0006FC04F81588569857A858B859C850E946E
:1016E000E40666C086E0FE013796DE0111960190A1
:1016F0000D928A95E1F7FF81E8856A857B85611502
:10170000710531F0EF3F31F481E0FF3F19F403C080
:1017100081E001C080E080FD4BC08091A70190E096
:101720009C012F5F3F4F277033274091A60150E067
:101730002417350709F443C0F983EA837D836C835A
:1017400066E070E00E949021DC01A855BE4F96E053
:10175000FE01319601900D929A95E1F72093A70131
:101760000E94D40825C090E066E070E00E949021BD
:1017700088559E4F0E947409882371F18091A601BB
:1017800090E066E070E00E949021FC01E855FE4F79
:101790004081518162817381848195810E94E40638
:1017A0008091A60190E00196877099278093A60109
:1017B0008091A6019091A7018913D5CF0DC00E94F9
:1017C000AE061092A7011092A601E8EDF1E086E0C6
:1017D000DF011D928A95E9F72C960FB6F894DEBFCB
:1017E0000FBECDBFDF91CF9108958091FE01859509
:1017F0008595859508958091FE0187700895909153
:10180000FE01977081E009F480E008958091210243
:10181000089590912102892B80932102089580954B
:101820009091210289238093210208951092210230
:10183000089590912002892B80932002089580952D
:101840009091200289238093200208951092200213
:1018500008958091FF01089508950C942C0C0C9428
:101860002D0C9091720292FD08C09091FF01981783
:1018700021F08093FF010C942F0C08958091FF01BB
:10188000882329F01092FF0180E00C942F0C08951A
:10189000CF93DF93E0910201F09103018091210247
:1018A0008083E0910201F0910301908180912002F8
:1018B000892B80838091FF01882381F0E0910201D0
:1018C000F09103019081892B808380910201909196
:1018D00003010E94321981110E943E0CC091020145
:1018E000D091030140E250E06EED71E0CE010E9424
:1018F0000A22892B69F080E2FE01AEEDB1E0019091
:101900000D928A95E1F7CE01DF91CF910C94DE180C
:10191000DF91CF9108950C942C0C9091720292FD5E
:1019200010C0982F990F990F990F692B6093FE01A2
:101930000E9466078091FE018595859585950C949A
:101940008B0C0C9466071092FE0180E00C948B0CBB
:101950002091FE01809582238093FE01982F97703D
:1019600099F430E0482F082E000C550B241735074A
:1019700059F09091720292FD07C0859585958595E5
:101980000E9487070C94A30C08959091720292FB19
:10199000222720F9281769F080FB92F990937202B0
:1019A00080917102909172020E940D0D82E00C9460
:1019B000A80C08958091720282FB882780F991E03B
:1019C00089270C94C50C81E00C94C50C80E00C9424
:1019D000C50C80E090E00E941F2221E0893E9E4FCE
:1019E00009F020E0822F089582E090E00C94172205
:1019F00083E090E00C941722CF9384E090E00E9463
:101A00001722C82F82E290E00E9417222C2F30E08C
:101A1000A901582BCA01CF910895CF93C92F682FE0
:101A200084E090E00E9425226C2F82E290E0CF912A
:101A30000C942522AB01BC018FE090E00C9437227E
:101A4000AB01BC0183E190E00C94372260E070E0D0
:101A5000CB010C94200D60E070E0CB010E941A0DC8
:101A60000C94260D69EE7EEF80E090E00E94432208
:101A700060E082E090E00E94252260E083E090E058
:101A80000E9425221092A2011092A3011092A4019B
:101A90001092A50160E084E090E00E94252260E0C1
:101AA00082E290E00E94252260E085E090E00E94C2
:101AB000252260E086E090E00E9425226FEF87E01B
:101AC00090E00E94252240E050E0BA0188E090E0DA
:101AD0000E94372260E08DE090E00E94252240E0E5
:101AE00050E0BA0188E190E00E94372260E087E18F
:101AF00090E00E94252240E050E0BA018CE190E0A5
:101B00000E94372260E070E080E290E00E94432271
:101B100040E050E0BA0188E190E00E9437220C9446
:101B20002B0D0C94320D682F8EE090E00C94252242
:101B30000E94971A60932B0270932C0280932D02BF
:101B400090932E02609327027093280280932902BB
:101B500090932A02089581E008950C94AB0D0895A6
:101B60000C94AF0D0C94AF0D0C94B20D0C94AF0D02
:101B70000C94B60D0C94AF0D88E790E10E94C81844
:101B80000E94BA0D0C94B80D0E94B00D0C94AF0DCC
:101B90000E947B100E946D020C947A160E94821A99
:101BA0000E9452110E94C80D0E94AE140C94B40DF4
:101BB0008F929F92AF92BF92CF92DF92EF92FF925D
:101BC0000F931F93CF93DF93CDB7DEB72A970FB64E
:101BD000F894DEBF0FBECDBF0E946711982E811111
:101BE0000E94980D82E2A82E82E0B82E00E010E05C
:101BF000802E802F0E949F10D82EF501C1905F018A
:101C0000C826B1F40F5F1F4F0530110589F78FEF1C
:101C100089838A831B820E948B1A8160782F9D831F
:101C20008C8349815A816B818D810E9489022FC0EA
:101C300080912F0281FD0E94A510E12CFF24F394D6
:101C40008C2D8F21F1F00E94AD0D882399F0EE824A
:101C50008F82DF2081E009F480E088870E948B1A60
:101C60008160782F9A8789874E815F8168858A8510
:101C70000E948902F801EE5DFD4F8081F826F08216
:101C800006C0E394FF0CF6E0EF12DACFBBCF81E0A1
:101C9000911001C080E02A960FB6F894DEBF0FBE07
:101CA000CDBFDF91CF911F910F91FF90EF90DF900B
:101CB000CF90BF90AF909F908F9008950E94D80DC5
:101CC0000E9479160E946E130C947E02CF93DF93CC
:101CD0000E94A10FEC01811521E5920708F045C093
:101CE000811530E5930708F094C0883E910528F5EA
:101CF000803E910508F001C1883A910570F4853A5B
:101D0000910508F07CC08130910509F475C008F494
:101D1000F1C0049708F0F1C0EDC08F3B910508F0C9
:101D2000E9C0C85AD0E0CC0FDD1FC65BDE4F09907A
:101D3000D881C02DCE019464E1C0811540E29407A2
:101D400058F4811551E0950708F0D7C08D3E9105F4
:101D500008F4D0C09065D2C0C11580E4D80708F45B
:101D6000C9C0DF70CE01906AC9C0811525E5920710
:101D7000A8F4811534E5930708F09EC0811543E56A
:101D8000940708F081C0811552E5950708F064C0FA
:101D9000D82FCC27CE01816F906AB0C0C11589E5DC
:101DA000D807A0F4C11528E5D20708F08BC0C115EB
:101DB00036E5D30708F09EC08C2F0E9435108F7136
:101DC00090E0D82FCC27CE01906298C0C1154AE58B
:101DD000D40708F47DC0CE0190568115904208F0DA
:101DE00089C08D2F8F710E943510DD27D0628F71D1
:101DF000AE01582BCA0182C081E090E07FC0C55A75
:101E0000D0E0C858DE4F8881C82FD0E0CE01906462
:101E100075C0F4E096958795FA95E1F7282F237021
:101E20003C2F337081E090E002C0880F991F3A95F3
:101E3000E2F79C68AC01522B9C2F9F70969596956B
:101E4000892F90E0EC01A5E0CC0FDD1FAA95E1F70A
:101E5000CA018C2B9D2B52C08370992721E030E062
:101E600002C0220F331F8A95E2F79C2F9695969514
:101E7000C92FD0E075E0CC0FDD1F7A95E1F7C22BBA
:101E8000D32BCE019C683AC08370992721E030E0C3
:101E900002C0220F331F8A95E2F79C2F96959695E4
:101EA000C92FD0E065E0CC0FDD1F6A95E1F7C22BAA
:101EB000D32BCE019A6822C0D82FCC27CE01846FB5
:101EC000906A1CC0DC2FCC27CE01806F906A16C0B0
:101ED0008C2F8F700E94351094E0D695C7959A95F7
:101EE000E1F7CF70D0E0DC2FCC27D0699E01282B02
:101EF000C90104C080E090E001C0CE01DF91CF9124
:101F00000895382F262F872F90E066E070E00E941A
:101F10009021FC01832F90E06EE170E00E949021FF
:101F20008E0F9F1FFC01E20FF11DEE0FFF1FE05609
:101F3000FF4F8591949108950E94810F0E94660E33
:101F400008958238910569F1B0F48133910509F45F
:101F50006DC048F48932910509F463C08A32910555
:101F600009F469C008958533910509F455C0893392
:101F70009105B9F00895833E910569F138F4803EEA
:101F80009105B1F0823E910509F10895863E9105D3
:101F9000A9F1873E9105B9F1843E910509F064C02D
:101FA00023C02091710220FD4FC021FD4DC0089536
:101FB0008091710280FD44C08091720280FF44C014
:101FC0008091710284FD42C083EE4DC08091710208
:101FD00082FF38C0F5CF8091710282FD33C08091BD
:101FE000720280FD31C0ECCF8091720281FF32C05D
:101FF0008091710284FD2AC087EE35C08091710204
:1020000083FF26C0F5CF8091710283FD21C08091AE
:10201000720281FD1FC0ECCF8091710285FD1CC052
:102020001DC08091710285FD19C016C0809171029A
:1020300086FD16C017C08091710286FD13C010C0C6
:1020400089E311C082EE0FC080EE0DC080E00BC0AE
:1020500086EE09C084EE07C089E205C085E303C0AF
:102060008AE201C081E390E008959091710292FFAD
:102070000DC0282F2871283019F4877F846006C08E
:10208000282F2471243011F48B7F886093FF0DC0BA
:10209000282F2871283119F4877E846106C0282FE3
:1020A0002471243111F48B7E88612091720220FF0B
:1020B0000DC0382F3871383019F4877F816006C021
:1020C000382F3171313011F48E7F886021FF0DC0BF
:1020D000282F2871283119F4877E816106C0282FA6
:1020E0002171213111F48E7E886194FD877E0895DF
:1020F00080E0089508950E94E90C811102C00E94B9
:10210000910D0E94F40C80932F020E94FC0C90937E
:102110007202809371020E947A100E94F80C682F5C
:1021200070E080E090E00E94060760919E0170914F
:102130009F018091A0019091A1010C943E07E82F8E
:10214000F0E0E858FD4F80810895089580EA8A956F
:10215000F1F7089500C008950C94A61008950C940A
:10216000AE100C94AF100C94AE100C94B310F89405
:10217000E82FE295EF70F0E031A1282F2F7081E079
:1021800090E001C0880F2A95EAF7982F9095932345
:1021900091A392A1892B82A3789408950F931F9302
:1021A000CF93DF93C1E8D1E089918F3F11F00E9476
:1021B000B71081E0C638D807B9F7CBE7D1E001E81E
:1021C00011E089918F3F11F00E94B7100C171D0785
:1021D000C1F7DF91CF911F910F910895CF92DF92B8
:1021E000EF92FF920F931F93CF93DF938C01C62F33
:1021F000D0E0CE018F579E4F7C01FC0190819F3F24
:1022000009F447C0D62EF894E92FE295EF70F0E07C
:1022100081A19F7021E030E001C0220F9A95EAF77A
:10222000822B81A382A12095282322A378940E9447
:10223000AA10EBE7F1E041E851E031E0C12C219137
:102240002F3F89F0A22FA295AF70B0E090968C91AD
:1022500090E02F7002C0959587952A95E2F780FD52
:1022600002C0832F01C080E0C82A330F4E175F07DA
:1022700031F7F70180818F3F11F00E94B71061E0C4
:10228000C11001C060E08D2D0E94AC10C00FD11FA5
:10229000C882DF91CF911F910F91FF90EF90DF9057
:1022A000CF9008950E94CE1085E0E8E7F2E0DF01CC
:1022B000982F1D929A95E9F7E3E7F2E0DF011D926E
:1022C0008A95E9F785E00E94AE110C94EC01FF922B
:1022D0000F931F93CF93DF9300D000D01F92CDB701
:1022E000DEB78E010F5F1F4F85E0F80111928A95CE
:1022F000E9F7F12C6F2DC8010E94EE10F394F5E080
:10230000FF12F8CF45E050E0B80183E792E00E9469
:102310000A22FF24F394009709F4F12C892B41F051
:1023200085E0F801A3E7B2E001900D928A95E1F70C
:102330002F2D45E068E772E083E792E00E94AF113D
:102340000E94EE018F2D0F900F900F900F900F9025
:10235000DF91CF911F910F91FF9008950895FF9203
:102360000F931F93CF93DF938C01F62ED72FC42F9B
:10237000222349F081E0809332020E948B1A9093CD
:10238000310280933002809132028823C1F0809123
:102390003002909131020E94A31A059780F0EF2D30
:1023A000FD2FD8014C2F50E0CD01801B910B8417DD
:1023B00095071CF48D918193F7CF10923202DF9133
:1023C000CF911F910F91FF9008950E948E1C0E9443
:1023D000CE0D0C949A1C0E949E1C0E945E0E0C94C2
:1023E000B81C0E94291A0E94751C0E94BC0D0E94F4
:1023F000E5110E94EB110E94C40DFBCF80913902C0
:1024000080FF06C06091090170E0660F771F2CC045
:1024100081FF08C06091090170E0660F771F660FA9
:10242000771F22C082FF09C06091090170E043E07C
:10243000660F771F4A95E1F717C06091380266234F
:10244000D1F020910801621778F78091090190E09E
:1024500070E033E0880F991F3A95E1F70E949021D0
:10246000622F70E00E94CE216038710540F4611542
:10247000710519F406C068E070E0862F08958FE7B3
:10248000089581E008958091390280FF08C060912D
:10249000050170E0759567957595679523C081FF77
:1024A00006C06091050170E0759567951BC082FFBD
:1024B00004C06091050170E012C06091370266238C
:1024C000A9F0209104016217A0F78091050170E046
:1024D00090E00E949021622F70E00E94CE2160382F
:1024E000710540F46115710519F406C061E070E0F2
:1024F000862F08958FE7089581E008958D3E21F499
:102500000E94FE11819504C08E3E29F40E94FE11A6
:1025100080933D0208958F3E21F40E94FE11819523
:1025200004C0803F29F40E94FE1180933C0208956C
:10253000893F19F40E94431205C08A3F31F40E947A
:102540004312819580933E0208958B3F21F40E94AF
:102550004312819504C08C3F29F40E94431280935A
:102560003F0208959FE0980F983078F421E030E022
:10257000A90102C0440F551F9A95E2F7CA01909134
:102580003B02892B80933B0208958D3F21F480917B
:10259000390281600BC08E3F21F480913902826044
:1025A00005C08F3F29F480913902846080933902FD
:1025B00008958D3E39F490913D0297FF35C01092F9
:1025C0003D0259C08E3E29F490913D021916BCF38C
:1025D0002BC090913C028F3E29F497FF25C01092AA
:1025E0003C0249C0803F19F41916CCF31DC09091EC
:1025F0003E02893F29F41916BCF410923E023BC0FA
:102600008A3F19F497FF10C0F8CF8B3F39F49091AF
:102610003F0297FF09C010923F022DC08C3F21F46A
:1026200090913F021916BCF39FE0980F983080F408
:1026300021E030E0A90102C0440F551F9A95E2F74E
:10264000CA01809590913B02892380933B0213C07D
:102650008D3F21F4809139028E7F0BC08E3F21F493
:10266000809139028D7F05C08F3F29F48091390216
:102670008B7F8093390280913C02811106C080914A
:102680003D02811102C01092380280913E028111F8
:1026900006C080913F02811102C010923702089556
:1026A0000E948B1A20913C02211104C020913D020E
:1026B000222321F0909336028093350220913E022E
:1026C000211104C020913F02222321F09093340273
:1026D000809333028AE392E00C94F818EF92FF9211
:1026E0000F931F93CF93DF9300D000D000D0CDB7CE
:1026F000DEB786E0EAE3F2E0DE01119601900D928A
:102700008A95E1F7E0903C02F0903D0200913E0294
:1027100010913F0210923C0210923D0210923E0234
:1027200010923F02E11003C0FF2009F464C08091C1
:102730003502909136020E94A31AFC0120913802C2
:10274000222339F080910A0190E08E179F0760F0F4
:1027500052C080910B0190E06AE070E00E949021ED
:102760008E179F0718F047C02F3F19F02F5F209357
:102770003802EE2061F00E94FE11682F1E1414F042
:102780008FEF01C081E00E94872180933C02FF20EF
:1027900061F00E94FE11682F1F1414F08FEF01C02A
:1027A00081E00E94872180933D0280913C02882332
:1027B00011F120913D022223F1F0082E000C990B1B
:1027C00065EB70E00E949021992319F090933C02F0
:1027D00003C081E080933C02822F220F990B65EBAE
:1027E00070E00E949021992319F090933D0203C05C
:1027F00081E080933D02011103C0112309F464C0FC
:1028000080913302909134020E94A31AFC0120911E
:102810003702222339F08091060190E08E179F073E
:1028200060F052C08091070190E06AE070E00E9481
:1028300090218E179F0718F047C02F3F19F02F5F88
:1028400020933702002361F00E944312682F101674
:1028500014F08FEF01C081E00E94872180933E0237
:10286000112361F00E944312682F111614F08FEFAC
:1028700001C081E00E94872180933F0280913E0247
:10288000882311F120913F022223F1F0082E000C41
:10289000990B65EB70E00E949021992319F09093B9
:1028A0003E0203C081E080933E02822F220F990BEB
:1028B00065EB70E00E949021992319F090933F02FC
:1028C00003C081E080933F0280913C0281110BC0E4
:1028D00080913D02811107C080913E02811103C0A9
:1028E00080913F0281110E945013EB82FC820D8384
:1028F0001E8386E0FE013196AAE3B2E001900D92BC
:102900008A95E1F726960FB6F894DEBF0FBECDBFCD
:10291000DF91CF911F910F91FF90EF900895EAE31F
:10292000F2E086E0DF011D928A95E9F71092380205
:102930001092370210923902089586E090E00C94CC
:102940001722682F86E090E00C94252280917D026A
:102950008470816280937D020C94A1140E94E90C22
:10296000811104C00E94910D0E94A6140E949D1422
:1029700080937D02282F26952695269530E02530D8
:10298000310524F08770806280937D0280917D0202
:1029900080FF04C086958695869501C080E00C94E2
:1029A000BF1520917D02822F869586958695482FAA
:1029B00050E04430510554F48F5F982F990F990FD0
:1029C000990F822F8770892B80937D0280917D02E1
:1029D000816080937D020E94A11480917D02869582
:1029E000869586950C94BF1580917D02982F9695BB
:1029F00096959695A1F0915E990F990F990F877012
:102A0000892B80937D02887F91E009F490E080918A
:102A10007D0290FB80F980937D020E94A114809139
:102A20007D028695869586950C94BF1580917D02D2
:102A300080FD13C0816080937D02813019F489E0AC
:102A400080937D0280917D020E94A11480917D027D
:102A50008695869586950C94BF15089580917D0284
:102A600080FF08C08E7F80937D020E94A11480E0C9
:102A70000C94BF15089580917D0280FD0C942E1555
:102A80000C94161590917D02892F869586958695D2
:102A90008F5F8F719770853038F4880F880F880F9B
:102AA000892B80937D0202C090937D0280917D02EC
:102AB000887F91E009F490E080917D0290FB80F99D
:102AC00080937D020E94A11480917D028695869557
:102AD00086950C94BF15853008F084E090917D02B6
:102AE0009770282F220F220F220F922B90937D0296
:102AF000987F21E009F420E090917D0220FB90F97D
:102B000090937D020C94BF150E946B1580917D02FD
:102B10000C94A1149C01FB018281882349F12E3B76
:102B2000FCE53F07C9F040F42C3BECE53E0769F0BB
:102B30002D3B3C4561F00895203C9CE5390791F020
:102B400070F0213C3C4589F0089584E001C080E0AC
:102B50000E94841580E008950E94F414FBCF0E9427
:102B6000D114F8CF0E943B15F5CF0E944215F2CF49
:102B700081E00895279A2F9808952F9808958F92AD
:102B80009F92AF92BF92CF92DF92EF92FF920F93FC
:102B90001F93CF93DF93C82F853050F4811109C064
:102BA00080918000877F809380000E94BD1506C0C1
:102BB000C4E08091800088608093800060918600EE
:102BC0007091870080E090E02C2F30E040E050E0F2
:102BD0000E94A1218B019C0142E036952795179513
:102BE00007954A95D1F7322F212F102F0027012F5B
:102BF000122F232F332780918600909187006CE05D
:102C000070E00E94BA216017710730F0C80169E0D6
:102C100070E00E94BA215CC080918600909187008C
:102C2000E0908600F0908700E0918600F0918700A8
:102C3000C6E0D0E0BE010E94BA21060F171F211D79
:102C4000311D4801590185E0880C991CAA1CBB1C48
:102C50008A95D1F7C701BE010E94BA216F01E12C0C
:102C6000F12CA7019601260F371F411D511DC501EB
:102C7000B4010E94E22169017A01C0918600D091DD
:102C80008700CA01B9010E94A1219E0140E050E0E5
:102C90000E94A121A70196010E94A121DC01CB0184
:102CA0002FE0B695A795979587952A95D1F700912E
:102CB00086001091870020E030E0081719072A07E6
:102CC0003B0728F46091860070918700CB01BC011E
:102CD00070938D0060938C00DF91CF911F910F91C5
:102CE000FF90EF90DF90CF90BF90AF909F908F902C
:102CF000089508950E94BA158AE08093800089E1C2
:102D0000809381008FEF9FEF9093870080938600E0
:102D10000C94AE14CF93DF93EC01FB0182818823E6
:102D200009F43CC1C430FDE5DF0760F4CB3F9CE50E
:102D3000D90788F49E0122503C452431310508F022
:102D40002EC109C0C236EDE5DE0729F0C63AFDE521
:102D5000DF0709F024C10E94FC0C9093720280935B
:102D60007102C1318CE5D80709F4C6C008F042C031
:102D7000C930ECE5DE0709F49BC000F5C5308CE5F1
:102D8000D80709F485C078F4C330ECE5DE0709F410
:102D900078C008F07AC0C230DC4509F0F5C08091F7
:102DA00071028160EFC0C7309CE5D90709F478C093
:102DB00008F07AC0809171028061E4C0CD30FCE5FA
:102DC000DF0709F487C058F4CB309CE5D90709F434
:102DD00079C008F07BC08091710288606FC0CF30ED
:102DE000FCE5DF0709F480C008F082C08091710221
:102DF000877FC8C0CE3F9CE5D90709F471C000F5B4
:102E0000C531FCE5DF0709F485C068F4C3319CE5F2
:102E1000D90709F475C008F095C00E94AE068091EC
:102E200071028F77AFC0CC3FFCE5DF07A9F108F056
:102E300054C0CB3FDC4509F0A7C08091720240C06E
:102E4000C230EDE5DE0709F489C058F4C1158DE5FF
:102E5000D80709F45AC008F069C0809172028260F4
:102E60002FC0C236EDE5DE0709F47CC0C63AFDE5A9
:102E7000DF0709F481C0C330DD4509F085C080E07B
:102E80006EC08091710282607DC08091710216C017
:102E900080917102886076C08091720282604FC01A
:102EA0008091710280626EC08091710280646AC0FC
:102EB0000E94AE0680917102806864C0846062C026
:102EC00081603DC0809171028E7F5CC080917102F3
:102ED0008D7F58C08091710216C08091720218C017
:102EE000809172028D7F2BC0809171028F7E4AC0CB
:102EF000809171028F7D46C0809171028F7B42C0AC
:102F000080917102877F8B7F3DC0809172028D7F9F
:102F10008E7F15C08091710282FB222720F991E0FB
:102F2000922790FB82F990FB83F92CC0809172026A
:102F3000982F909591708E7F892B90FB81F98093CB
:102F4000720222C00E94AE068091710287FB222786
:102F500020F991E0922790FB87F914C081E00E944C
:102F6000930D12C08091710284FB222720F991E019
:102F7000922790FB84F906C080917102982F90955A
:102F800090FB80F98093710280917102909172029E
:102F90000E940D0D0E94AE0680E001C081E0DF912D
:102FA000CF910895CF93DF9386319C4541F5EB0196
:102FB0000E94060C982F8A81209102013091030112
:102FC000882379F09A7A81E009F480E080934002C6
:102FD000911102C069E201C065E3C9010E94C819EC
:102FE0000AC080914002811102C069E201C065E31C
:102FF000C9010E94D3190E94480C80E001C081E001
:10300000DF91CF9108950F931F93CF93DF93C42F38
:10301000D22FFC0182818823C9F0409343020E9491
:103020008B1A909342028093410280E28C0F883089
:1030300008F057C0C77081E001C0880FCA95EAF751
:10304000DF91CF911F910F910C940B04809143025B
:10305000481330C080914102909142020E94A31A0D
:10306000883C910538F510E21D0FCD17B9F080E2CC
:103070008C0F883040F4C77081E001C0880FCA957A
:10308000EAF70E941204183028F581E09D2F97700E
:1030900001C0880F9A95EAF70E940B04802F0E94C6
:1030A00002041830F0F4D77081E001C0880FDA957F
:1030B000EAF70AC080E28C0F883098F4C77081E08C
:1030C00001C0880FCA95EAF7DF91CF911F910F9148
:1030D0000C941204802FDF91CF911F910F910C94CB
:1030E0000204DF91CF911F910F9108950F939C01DE
:1030F000CB01243F4CE5340731F188F4293DFCE550
:103100003F07D9F02A3D4CE5340779F1283D3C458D
:10311000A9F506E221EE41EE68ED7CE52BC0263FE5
:10312000FCE53F07E1F0A8F0273F3C4539F507E211
:1031300025EE46EE67EF7CE51DC007E225EE45EE85
:1031400069ED7CE517C006E221EE40EE64EF7CE518
:1031500011C007E225EE44EE65EF7CE50BC006E208
:1031600021EE42EE66EF7CE505C008E221E045EE87
:103170006AED7CE50E94031880E008C0FC018281B2
:10318000882319F01092430201C081E00F91089545
:1031900090938701809386010895909349028093CC
:1031A00048020895E0914802F0914902309721F0D9
:1031B0000190F081E02D099480E00895E0914802AB
:1031C000F0914902309799F020911801222359F08B
:1031D0002091710227FF07C0DC012C9111962C93DE
:1031E000119726E02C930280F381E02D0994089535
:1031F000E0914802F0914902309739F022E0DC0179
:103200002C930480F581E02D0994089520914602C5
:10321000309147022817390771F090934702809345
:103220004602E0914802F0914902309721F0068071
:10323000F781E02D099408952091440230914502D0
:103240002817390771F09093450280934402E0916A
:103250004802F0914902309721F00084F185E02D79
:1032600009940895FC01329680911801882331F069
:103270008091710287FF02C09EE101C096E080E06C
:10328000915028F021912223D9F38F5FF9CF08952F
:10329000662351F1209118012223E9F02091710257
:1032A00027FF19C0462F4695469546954E31E0F4C6
:1032B000677021E030E002C0220F331F6A95E2F709
:1032C000FC01E40FF11D828190E02823392381E085
:1032D000232B69F409C0FC013296089621916217EC
:1032E00029F0E817F907D1F780E0089581E0089503
:1032F0009C01FC0132969FEF80E04191461789F0D6
:103300009F3F19F4411101C0982F8F5F8630A9F7B4
:103310009F3F39F0F901E90FF11D97FDFA9562839E
:10332000089508959C012A5F3F4FFC014281461396
:1033300001C01282019682179307B9F70895262FCC
:103340002695269526952E3168F4FC01E20FF11D95
:10335000677021E030E001C0220F6A95EAF78281B0
:10336000282B22830895262F2695269526952E31E3
:1033700070F4FC01E20FF11D677021E030E001C044
:10338000220F6A95EAF720958281282322830895E7
:1033900020911801222329F02091710227FD0C941D
:1033A0009F190C94781920911801222329F020915B
:1033B000710227FD0C94B3190C94921920911801F5
:1033C000FC013296222331F08091710287FF02C006
:1033D0008EE101C086E0DF011D928A95E9F708952C
:1033E00008950C94F01983E080934A020C94F1192B
:1033F000811102C081E001C082E080934A020C94F6
:10340000F1190C94F81981E080934A020C94F11997
:103410000C94031A08950C940A1A0C940B1A0C9429
:103420000A1A0C940A1A0C940A1ACF930E94111AC1
:103430000E9467110E940F1AC0E08C2F0E949F10FB
:10344000811104C0CF5FC530C1F701C081E0CF91C9
:10345000089508951F920F920FB60F9211248F9323
:103460009F93AF93BF9380914B02811113C08091C2
:103470007E0290917F02A0918002B09181024196DC
:10348000A11DB11D80937E0290937F02A0938002C4
:10349000B0938102BF91AF919F918F910F900FBE1A
:1034A0000F901F90189580918602843031F10E9410
:1034B000590210924B0220E488E190E00FB6F89494
:1034C000A895809360000FBE2093600083B7817F32
:1034D000846083BF83B7816083BF7894889583B706
:1034E0008E7F83BF0FB6F894A895809160008861A5
:1034F00080936000109260000FBE08950E94AE0697
:103500000C94600282E084BD93E095BD9AEF97BD74
:1035100080936E0008952FB7F89480917E02909169
:103520007F02A0918002B09181022FBF08952FB732
:10353000F89460917E0270917F0280918002909158
:1035400081022FBF08959C014FB7F89480917E02AD
:1035500090917F02A0918002B09181024FBF821BA7
:10356000930B089578941F920F920FB60F92112427
:103570008F939F93AF93BF9380917E0290917F0230
:10358000A0918002B09181020196A11DB11D80938E
:103590007E0290937F02A0938002B0938102BF913C
:1035A000AF919F918F910F900FBE0F901F90189524
:1035B00081E08093E00080E28093D8001092C900FF
:1035C0008FE19EE40197F1F700C0000087E090EBE7
:1035D000DC0180938F0290939002A0939102B093AC
:1035E00092029CE088E10FB6F894A8958093600061
:1035F0000FBE90936000FFCF80916F0208950895F1
:1036000022E02093E9002FEF3091E800215035FDB2
:1036100006C035ED3A95F1F700002111F5CF209164
:10362000E80025FF0BC040E050E066E070E00E943B
:103630002A1D8091E8008E778093E8000895CF934B
:10364000DF9320911801222339F02091710227FF86
:1036500003C060E222E002C068E021E02093E900BC
:103660002FEF3091E800215035FD06C035ED3A9539
:10367000F1F700002111F5CF2091E80025FF1DC0D2
:10368000EC0180911801811105C040E050E068E034
:1036900070E003C070E040E050E0CE010E942A1DBF
:1036A0008091E8008E778093E80080E2FE01AFE42D
:1036B000B2E001900D928A95E1F7DF91CF910895E4
:1036C00080934C0270934E0260934D02809186026B
:1036D000843001F582E08093E9008FEF9091E8005B
:1036E000815095FD06C095ED9A95F1F70000811186
:1036F000F5CF8091E80085FF0DC040E050E063E029
:1037000070E08CE492E00E942A1D8091E8008E77A0
:103710008093E8000895BC0184E00C94601BBC0118
:1037200083E00C94601B0C94081A6091820281E083
:10373000611101C080E00C94F3199091860281E040
:10374000943009F080E0609182020C94F81942E014
:1037500061EC81E00E942E1E42E261EC82E00E9458
:103760002E1E9091860281E0943009F080E06091F5
:1037700082020C94011A80918802833009F45DC0A2
:1037800030F4813071F0823009F496C008958A30A7
:1037900009F482C08B3009F468C0893009F0A4C0F4
:1037A00020C080918702813A09F09EC08091E80094
:1037B000877F8093E80080918B0290918C02892B07
:1037C00021F460E28FE492E003C060E080E090E0EA
:1037D00070E00E94751D8091E8008B778093E8006F
:1037E000089580918702813209F07EC080918B021A
:1037F00090918C02029708F077C08091E800877F53
:103800008093E8008091E80082FD05C080918602E7
:103810008111F8CF69C08091F200823031F480913B
:10382000F100813011F0863021F48091F100809315
:103830006F028091E8008B7753C080918702813AB4
:1038400009F052C080918B0290918C02892B09F073
:103850004BC08091E800877F8093E8008091E8006A
:1038600080FFFCCF8091180136C0809187028132A1
:10387000D9F580918B0290918C02892BA9F58091CA
:10388000E800877F8093E8000E94631E8091890290
:10389000809318010C94AE0680918702813221F545
:1038A0008091E800877F8093E8000E94631E8091EA
:1038B0008A0280937002089580918702813AA1F470
:1038C0008091E800877F8093E8008091E80080FF86
:1038D000FCCF809170028093F1008091E8008E7798
:1038E0008093E8000C94631E089584B7877F84BF9B
:1038F0000FB6F894A895809160008861809360006D
:10390000109260000FBE90E080E80FB6F8948093AC
:103910006100909361000FBE0C94031A0E94B51EC3
:103920000E94081FE2EEF0E080818460808378943A
:103930000C946C218CE091E00C94CD18809186025F
:103940008530A9F480918602853079F40E94531A5B
:10395000809184028823B1F30E94151A882391F381
:103960000E94141D0E94AE06EDCF0C947E1A08959D
:1039700008950C94BB1C292F332723303105C9F03F
:1039800060F42130310581F02230310509F044C066
:103990008BE390E02CE731E043C021323105E1F0C8
:1039A0002232310549F138C082E190E027EB31E065
:1039B00037C099278130910549F028F0029761F5C9
:1039C000E4E5F1E005C0E8E7F1E002C0E6E6F1E099
:1039D000849190E09F0124C06115710541F0613030
:1039E0007105D1F489E090E027EA31E019C089E05F
:1039F00090E02EE831E014C06115710541F06130AE
:103A0000710551F486EB90E029EC31E009C080E4C7
:103A100090E02FE732E004C080E090E020E030E06A
:103A2000FA0131832083089584E089BD86E089BD51
:103A300009B400FEFDCF8091D8008F7D8093D8001F
:103A40008091E00082608093E0008091E00081FD41
:103A5000FCCF0895CF92DF92EF92FF920F931F93C6
:103A6000CF93DF93EC018B017A010E94821E8111BA
:103A700033C0E114F10439F0F70180819181081B12
:103A8000190BC80FD91FC12CD12C0115110519F123
:103A90008091E80085FD16C08091E8008E778093C4
:103AA000E800E114F10449F0F70180819181C80E2A
:103AB000D91ED182C08285E00FC00E94821E882359
:103AC00021F30AC089918093F10001501109FFEFA1
:103AD000CF1ADF0ADACF80E0DF91CF911F910F91EB
:103AE000FF90EF90DF90CF90089520918D0230915C
:103AF0008E022617370748F06115710539F42091B9
:103B0000E8002E772093E80001C0B901FC0120E015
:103B10006115710561F1809186028823D9F18530A4
:103B2000D9F18091E80083FD39C08091E80082FDE1
:103B30002BC08091E80080FFEBCF8091F20090E0F5
:103B40006115710551F08830910538F42191209369
:103B5000F100615071090196F3CF21E0089709F057
:103B600020E08091E8008E778093E800D1CF21118A
:103B7000D2CF0AC080918602882361F0853061F03F
:103B80008091E80083FD0AC08091E80082FFF2CFB7
:103B900080E0089582E0089583E0089581E008952B
:103BA00020918D0230918E022617370748F061155B
:103BB000710539F42091E8002E772093E80001C0C8
:103BC000B901FC0120E06115710579F1809186024F
:103BD000882309F43DC0853009F43CC08091E80099
:103BE00083FD3AC08091E80082FD2CC08091E800FE
:103BF00080FFE9CF8091F20090E06115710559F0E6
:103C00008830910540F424912093F1003196615061
:103C100071090196F2CF21E0089709F020E0809128
:103C2000E8008E778093E800CECF2111CFCF0AC075
:103C300080918602882361F0853061F08091E800F0
:103C400083FD0AC08091E80082FFF2CF80E00895F2
:103C500082E0089583E0089581E00895982F9530DB
:103C600068F59093E900981739F07091EC00209175
:103C7000ED005091F00003C0242F762F50E021FD7D
:103C800002C09F5FECCF3091EB003E7F3093EB00A2
:103C90003091ED003D7F3093ED003091EB003160CD
:103CA0003093EB007093EC002093ED005093F00004
:103CB0002091EE0027FDE5CF80E008958F7080937E
:103CC000E90081E008958091870287FF11C080910B
:103CD000E80082FD05C0809186028111F8CF11C0F5
:103CE0008091E8008B770BC080918602882349F091
:103CF0008091E80080FFF8CF8091E8008E77809374
:103D0000E80008952091E4003091E50095E64091A7
:103D1000EC00842F817040FF23C08091E80080FD7B
:103D20001DC080918602882399F0853099F080919A
:103D3000EB0085FD11C04091E4005091E50024178F
:103D4000350729F3915011F09A01E1CF84E00895ED
:103D500082E0089583E0089581E0089580E0089569
:103D60004091E80042FFDDCF08950E94121F0E949B
:103D7000151FE0EEF0E0808181608083E8EDF0E0E7
:103D800080818F77808319BCE3E6F0E080818160D9
:103D900080831092850208950E94121F0E94151FB1
:103DA0008091D8008F778093D8008091D800806868
:103DB0008093D8008091D8008F7D8093D80084E0D4
:103DC00089BD86E089BD09B400FEFDCF1092860250
:103DD00010928202109284021092830242E060E00C
:103DE00080E00E942E1E8091E1008E7F8093E10092
:103DF0008091E20081608093E2008091E20088601F
:103E00008093E2008091E0008E7F8093E00008952F
:103E1000E3E6F0E080818E7F808381E080938502FD
:103E20000C94CC1E1092E20008951092E1000895C7
:103E30001F920F920FB60F9211242F933F934F931F
:103E40005F936F937F938F939F93AF93BF93EF9302
:103E5000FF938091E10082FF0BC08091E20082FF1E
:103E600007C08091E1008B7F8093E1000E946B216D
:103E70008091E10080FF19C08091E20080FF15C0B1
:103E80008091E2008E7F8093E2008091E200806169
:103E90008093E2008091D80080628093D80019BCA2
:103EA00085E0809386020E94951B8091E10084FF4B
:103EB00030C08091E20084FF2CC084E089BD86E0A0
:103EC00089BD09B400FEFDCF8091D8008F7D80931D
:103ED000D8008091E1008F7E8093E1008091E20024
:103EE0008F7E8093E2008091E20081608093E20007
:103EF00080918202882311F084E007C08091E30062
:103F000087FD02C081E001C083E0809386020E94A9
:103F10009D1B8091E10083FF29C08091E20083FF17
:103F200025C08091E100877F8093E10082E080934B
:103F30008602109282028091E1008E7F8093E100E0
:103F40008091E2008E7F8093E2008091E2008061A8
:103F50008093E20042E060E080E00E942E1E8091AB
:103F6000F00088608093F0000E94931BFF91EF9116
:103F7000BF91AF919F918F917F916F915F914F9181
:103F80003F912F910F900FBE0F901F9018951F9289
:103F90000F920FB60F9211242F933F934F935F937D
:103FA0006F937F938F939F93AF93BF93CF93DF9341
:103FB000EF93FF93C091E900CF708091EC00D82F70
:103FC000D17080FDD0E81092E9008091F000877FE9
:103FD0008093F00078940E940B201092E900809169
:103FE000F00088608093F000CD2BCF70C093E90083
:103FF000FF91EF91DF91CF91BF91AF919F918F9101
:104000007F916F915F914F913F912F910F900FBED4
:104010000F901F9018951F93CF93DF93CDB7DEB706
:10402000AA970FB6F894DEBF0FBECDBFE7E8F2E067
:104030008091F100819322E0EF38F207C9F70E94E6
:10404000BB1B8091E80083FF2EC180918702909175
:104050008802492F50E04A30510508F024C1FA0186
:10406000EA5BFF4F0C940422803821F0823809F07B
:104070001AC108C08091830290918402992389F02B
:1040800082600FC080918B028F70853008F00BC169
:104090008093E9008091EB0085FB882780F91092DE
:1040A000E9009091E800977F9093E8008093F100F9
:1040B0001092F100D1C0282F2D7F09F0F4C0882381
:1040C00019F0823061F0EFC080918902813009F0EF
:1040D000EAC0933009F080E0809384022EC0809182
:1040E000890281112AC080918B028F702FEF280FD7
:1040F000243008F0D8C08093E9002091EB0020FF25
:104100001CC0933021F48091EB00806214C0909128
:10411000EB0090619093EB0021E030E0A90102C038
:10412000440F551F8A95E2F74093EA001092EA0087
:104130008091EB0088608093EB001092E900809101
:10414000E800877F8093E8000E94631EACC0811165
:10415000AAC0109189021F778091E3008078812B9B
:104160008093E3008091E800877F8093E8000E94BD
:10417000631E8091E80080FFFCCF8091E30080689F
:104180008093E300111102C082E001C083E08093BC
:10419000860289C08058823008F085C080918902EB
:1041A00090918A028C3D53E0950779F583E08A83EC
:1041B0008AE289834FB7F894DE01139620E03EE04F
:1041C00051E2E32FF0E050935700E49120FF03C049
:1041D000E295EF703F5FEF708E2F90E0EA3010F0C5
:1041E000C79601C0C0968D939D932F5F243149F7E8
:1041F0004FBF8091E800877F8093E8006AE270E01B
:10420000CE0101960E94751D16C060918B027091BF
:104210008C02AE014F5F5F4F0E94B91CBC01892B1D
:1042200009F441C09091E800977F9093E80089815C
:104230009A810E94D01D8091E8008B778093E800DE
:1042400032C0803881F58091E800877F8093E80054
:10425000809182028093F1008091E8008E7772CF86
:10426000811121C08091890290918A029927029739
:10427000D4F48091E800877F8093E80080918902E0
:10428000809382020E94631E80918202811106C087
:104290008091E30087FD02C081E001C084E080934B
:1042A00086020E94A71B8091E80083FF0AC08091CC
:1042B000E800877F8093E8008091EB008062809324
:1042C000EB00AA960FB6F894DEBF0FBECDBFDF910C
:1042D000CF911F9108950895CF93809186028823EE
:1042E000A1F0C091E900CF709091EC00892F81700E
:1042F00090FD80E8C82B1092E9008091E80083FDD2
:104300000E940B20CF70C093E900CF910895002444
:1043100080FD060E660F11F08695D1F7802D089569
:104320000024552704C0080E591F880F991F0097B5
:1043300029F076956795B8F37105B9F7802D952F1B
:104340000895EE27FF27AA27BB2708C0A20FB31F97
:10435000E41FF51F220F331F441F551F96958795A5
:104360007795679598F37040A9F7009799F7BD0185
:10437000CF010895AA1BBB1B51E107C0AA1FBB1F99
:10438000A617B70710F0A61BB70B881F991F5A95E1
:10439000A9F780959095BC01CD01089597FB072E54
:1043A00016F4009407D077FD09D00E94BA2107FCCB
:1043B00005D03EF4909581959F4F08957095619535
:1043C0007F4F0895A1E21A2EAA1BBB1BFD010DC051
:1043D000AA1FBB1FEE1FFF1FA217B307E407F507B5
:1043E00020F0A21BB30BE40BF50B661F771F881F91
:1043F000991F1A9469F760957095809590959B0127
:10440000AC01BD01CF010895EE0FFF1F0590F4919F
:10441000E02D0994FB01DC0104C08D91019080190D
:1044200021F441505040C8F7881B990B0895F99921
:10443000FECF92BD81BDF89A992780B50895A8E175
:10444000B0E042E050E00C944B22262FF999FECFC9
:1044500092BD81BDF89A019700B4021639F01FBAD7
:1044600020BD0FB6F894FA9AF99A0FBE08950396F4
:10447000272F0E9426220E942522252F0E942622D5
:10448000242F0C9426220196272F0E9426220C947A
:104490002522DC01CB01FC01F999FECF06C0F2BD5B
:1044A000E1BDF89A319600B40D9241505040B8F7F2
:0644B0000895F894FFCF0F
:1044B600C8000002280850011E0A1401FC1A1F1B1E
:1044C600001B8F1B8B1BFF1A01E200E900EA00B5F7
:1044D60000B600B700CD008301CC008A019201949A
:1044E600012102230224022502260227022A02B300
:1044F60000B4006F007000818283E200E900EA00E8
:10450600B500B600B700CD008301CC008A01920148
:1045160094012102230224022502260227022A02EE
:10452600B300B4006F007000818283336766929196
:06453600906535329593FB
:00000001FF
